:10000000000002308A004A2AFF0003088301FE0034
:100010000408FC000A08FD0004308A00C22CA80174
:10002000B900BA01A01128080319A0150530A700CE
:100030002730B600103028200330B600E8302820E2
:10004000B60164302820B6010A30282039082F284C
:10005000B5003A08B2003908B100A0213108B1005A
:10006000A7030319A0112808031939282702031828
:1000700040283108031DA011A0194028303E8028D7
:100080000800BD0022088400AA01F030AA0508304B
:10009000BE0003100318AA0A5C20BD0CBE0B4A2840
:1000A0000000C21A2A0C5C20552803145C20260884
:1000B000B6002508E720452A8413C21F6B280008D4
:1000C0002904421F29068000841700082904031C04
:1000D00029068000762800082904031C2906421BF3
:1000E00029068000841729098005762842081F39CF
:1000F000FF3EB2004108F53E0318B20A0000F428A2
:10010000A11A412808000821A20084178004841342
:10011000B501311CB50092200319452A922003191C
:10012000452A92282208B5060130B100B201000824
:1001300022053506031D0800B10A0319B20F9728DE
:10014000080003178D00031783168C130C148312F9
:100150000C088D0A452A03178C0083168C130C1586
:1001600055308D00AA308D008C148C18B5280C11D8
:1001700083128D0A452A83178001840AFF3E031DDE
:10018000BC28452A0830BD002A18DE212308840037
:1001900024082A193D222A1D3F2222088400290909
:1001A0008417800522088400B20CB10C00082904D1
:1001B000031C29068000DF20BD0BD228452A230816
:1001C000840024088006000080060800B601B500FF
:1001D000FF30B507031CB607031C452A0330B200E5
:1001E000DF30F420E828B201E83EB100B209FC306B
:1001F000031CFD28B1070318FA28B1070000B20F4D
:10020000FA2831180329B11C072900000729080022
:10021000BF000630BF190730840001308A003F0854
:10022000073982070134023404340834103420348E
:1002300040348034013EA6000A30B900BA01BB0147
:10024000BC012621A60B1C293908080034083C06ED
:100250008039BE00B41F3729B109B209B309B40906
:10026000B10A0319B20A0319B30A0319B40ABC1F6D
:100270004429B909BA09BB09BC09B90A0319BA0A60
:100280000319BB0A0319BC0AB501B601B701B801CD
:10029000C701C801C901CA013C083B043A0439043A
:1002A000031982292030BD000310B10DB20DB30D2A
:1002B000B40DC70DC80DC90DCA0D3C084A02031D77
:1002C0006B293B084902031D6B293A084802031DAC
:1002D0006B2939084702031C7C293908C7023A08F0
:1002E000031C3A0FC8023B08031C3B0FC9023C0821
:1002F000031C3C0FCA020314B50DB60DB70DB80DA3
:10030000BD0B5429BE1F8F29B509B609B709B80915
:10031000B50A0319B60A0319B70A0319B80A470838
:10032000B9004808BA004908BB004A08BC003508B3
:10033000B1003608B2003708B3003808B400452AC7
:10034000BA01B9011030BD00320DB90DBA0D350832
:10035000B9023608031C360FBA020318B62935084D
:10036000B90736080318360FBA070310B10DB20DDE
:10037000BD0BA4293108452A2030BD00C701C801A2
:10038000C901CA010310311CD3293908C7073A082B
:1003900003183A0FC8073B0803183B0FC9073C086E
:1003A00003183C0FCA07CA0CC90CC80CC70CB40C04
:1003B000B30CB20CB10CBD0BC2290800B501B601DB
:1003C000E529B20CB10CB50DB60DFF3E0318E129BD
:1003D0003608B2003508B100452AB100B41BF2213D
:1003E0003108452AB109B209B309B409B10A0319A0
:1003F000B20A0319B30A0319B40A0800B10106309E
:10040000841384000230842000303202031C182A36
:10041000031D0E2AC8303102031C182A0130320293
:10042000031C1D2A031D182A0E303102031C1D2A2D
:10043000FF30B200B1000314452A0B30AA00BA11F4
:10044000B1010230842000303202031C2D2A031D2A
:100450002C2A5A3031020318BA150310BA0CB90C01
:10046000AA0B1F2A7F303905B1000310B90D3A0DD0
:100470001F39B20031080310452A8004422AFF3A8E
:100480008005432AFF3A84178005831383120313E0
:1004900000000800A001073083169C0007309F0071
:1004A00007309C00FF308500FE3086008701880100
:1004B000FF3088008813831288130830A200203090
:1004C000A9000830A3004030A4000130AA00B10107
:1004D0008A01C220B1018A01C220831688138312C7
:1004E000881764308A01E6205B10DB1400308A0133
:1004F000A120D40005305407D50001308A01A12085
:1005000001390319DB12031DDB168A110A12DB1EE7
:100510009C2A0A308A01A120DE0005308A01A12030
:10052000E10006308A01A120DF0007308A01A12006
:10053000E0008A110A129D2ADB120B308A01A120E9
:10054000013903195B12031D5B160830A20010303D
:10055000A9000130C2008C30C100A601A5012030E5
:10056000A10030308A01412031308A0141203230EF
:100570008A01412033308A01412034308A014120F0
:1005800035308A01412036308A01412037308A01D6
:10059000412038308A01412039308A0141202E30F3
:1005A0008A0141202E308A0141202E308A014120CB
:1005B0000D308A0141200A308A0141200830A20012
:1005C0001030A9000130C2008C30C100A601A50185
:1005D0002030A10050308A01412047308A0141205B
:1005E00041308A01412032308A01412033308A0172
:1005F000412031308A01412078308A014120203069
:100600008A0141204B308A0141206F308A0141200C
:100610006E308A01412074308A01412072308A0193
:1006200041206F308A0141206C308A0141206330C3
:100630008A01412075308A01412020308A01412001
:100640004B308A01412061308A01412072308A0199
:10065000412074308A01412069308A0141202030D4
:100660008A0141202F308A01412020308A01412017
:1006700048308A01412061308A0141207A308A0164
:10068000412061308A01412072308A0141202030AE
:100690008A0141204B308A01412061308A0141208A
:1006A00072308A01412061308A01412062308A0122
:1006B000412061308A01412079308A014120203077
:1006C0008A0141202F308A01412020308A014120B7
:1006D00032308A01412030308A01412031308A0194
:1006E000412030308A0141200D308A0141200A30FA
:1006F0008A01412056308A01412065308A0141201B
:1007000072308A01412073308A01412069308A01A8
:10071000412079308A0141206F308A0141206E30BA
:100720008A0141203A308A01412020308A0141204B
:1007300031308A0141202E308A01412033308A0134
:1007400041202E308A01412030308A0141202E3054
:100750008A01412036308A01412030308A0141200F
:100760000D308A0141200A308A01412053308A012C
:10077000412069308A01412073308A014120743060
:100780008A01412065308A0141206D308A01412073
:1007900020308A01412068308A01412061308A017D
:1007A00041207A308A01412069308A01412072302B
:1007B0008A0141202E308A0141200D308A014120DA
:1007C0000A308A0141208A110A12DB1E982C083057
:1007D000A2001030A9000130C2008C30C100A60177
:1007E000A5012030A10055308A0141207A308A01CC
:1007F000412061308A0141206B308A0141207430F0
:100800008A01412061308A0141206E308A014120F5
:1008100020308A0141206B308A01412075308A01E5
:1008200041206D308A01412061308A0141206E30C3
:100830008A01412064308A01412061308A014120CF
:1008400020308A0141206B308A0141206F308A01BB
:10085000412064308A0141206C308A01412061309E
:100860008A01412072308A01412069308A01412089
:1008700020308A01412062308A01412065308A019E
:1008800041206C308A0141206C308A014120653062
:100890008A0141206B308A01412074308A01412055
:1008A00065308A01412020308A01412062308A016E
:1008B000412075308A0141206C308A014120753019
:1008C0008A0141206E308A01412064308A01412032
:1008D00075308A0141202C308A01412020308A0164
:1008E000412055308A0141204B308A01412020307F
:1008F0008A01412064308A01412065308A0141200B
:1009000076308A01412072308A01412065308A01A7
:10091000412064308A01412065308A0141202E3017
:100920008A0141200D308A0141200A308A0141208C
:10093000AC01AB018A110A12BF2C04302C078A00CB
:10094000A8302B0703188A0AAB0A0319AC0A8200E5
:100950003F3406345B344F3466346D347D340734B1
:100960007F346F3477347C3439345E347934713485
:1009700063345C34403436347334703400348A1158
:100980000A1641288A110A120B1CE62C86080B1045
:100990008A110A12061FD02CD80A8A110A12D12CE9
:1009A000D8018A110A12861FD92CD90A8A110A1273
:1009B000DA2CD9018A110A12861EE22CDA0A8A116F
:1009C0000A12E32CDA018A110A12072D8A110A127F
:1009D0005B1C072D571CF02C08144C088811012DA6
:1009E000D71CF62C88154D080811012D571DFC2C1D
:1009F00008154E088810012DD71D012D88144F08A9
:100A00000810870001300310D70D571AD7008A113C
:100A10000A125B19B22DD8088A110A120319562D31
:100A2000643058028A110A12031C352D6E305802A8
:100A30008A110A12031C312D540A8A110A12031951
:100A40002C2D8A110A125B1C2C2DD40A8A110A1231
:100A5000BC258A110A1249276430D8008A110A126B
:100A6000322DD80A8A110A12562D013058028A11E5
:100A70000A12031D552D540A8A110A1203194B2D0F
:100A80008A110A125B1C4B2DD40A8A110A12BC254A
:100A90008A110A1249271430DC008A110A16E7204D
:100AA0000230D8008A110A12562DD80AD9088A11A4
:100AB0000A120319A12D643059028A110A12031C6B
:100AC000802D6E3059028A110A12031C7C2DD40825
:100AD0008A110A120319772D8A110A125B1C772DCD
:100AE000D4038A110A12BC258A110A1249276430DC
:100AF000D9008A110A127D2DD90A8A110A12A12D54
:100B0000013059028A110A12031DA02DD4088A113E
:100B10000A120319962D8A110A125B1C962DD40312
:100B20008A110A12BC258A110A1249271430DC00E6
:100B30008A110A16E7200230D9008A110A12A12D63
:100B4000D90ADA088A110A120319B22D64305A023E
:100B50008A110A12031CB12DDA01DB158A110A125F
:100B6000B22DDA0A0B117D088A007C0884007E0809
:100B70008300FF0E7F0E090054085502031D01304B
:100B8000CB000301DB1801304B048A110A12031950
:100B9000482FDB105408FF3CC3000030031CFF3E0D
:100BA000C400C5018A110A12C41FD72DC503450808
:100BB000C600B401B301B2010530B1004608BC0063
:100BC0004508BB004408BA004308B9008A01BC21AB
:100BD0003408D3003308D2003208D1003108D000E5
:100BE000BC01BB010130BA003B30B90050083902EA
:100BF000BD003A08BE005108031C510FBE023B085D
:100C0000BF005208031C520FBF023C08C00053082B
:100C1000031C530FC0023D08D0003E08D1003F081E
:100C2000D2004008D3008A110A12D31B3F2E003095
:100C300053028A110A12031C3F2E8A110A12031D45
:100C40003B2E003052028A110A12031C3F2E8A11D9
:100C50000A12031D3B2E003051028A110A12031C96
:100C60003F2E8A110A12031D3B2E003050028A11BA
:100C70000A12031C3F2ECF018A110A12452EAC0125
:100C80001230AB008A019D24CF005308B4005208F3
:100C9000B3005108B2005008B100BC01BB01BA0159
:100CA0000A30B9008A0126213C08B0003B08AF0099
:100CB0003A08AE003908AD0030082F042E042D0488
:100CC0008A110A12031DC12E5308B4005208B30042
:100CD0005108B2005008B100BC01BB01BA010A3092
:100CE000B9008A0126213408D3003308D200320823
:100CF000D1003108D0005308B4005208B3005108A5
:100D0000B2005008B10000308A011A21AC01AB00DA
:100D10008A019D24AD0080302D07CD005308B4001A
:100D20005208B3005108B20050088A01ED21AD000D
:100D30003208AE00AE088A110A12031DA92E0A302D
:100D40002D028A110A120318A92ECE018A110A1245
:100D5000B92E5308B4005208B3005108B20050082D
:100D6000B10001308A011A21AC01AB008A019D2437
:100D7000CE00AC01AB018A019D24CC008A110A127D
:100D8000482F5308B4005208B3005108B20050086D
:100D9000B10000308A011A21AC01AB008A019D2408
:100DA000CC005308B4005208B3005108B2005008F8
:100DB0008A01ED21AD003208AE00AE088A110A1298
:100DC000031D0A2F0A302D028A110A1203180A2F56
:100DD0005308B4005208B3005108B20050088A0109
:100DE000ED21AD003208AE002D08053A2E048A111F
:100DF0000A12031D062FAC01AB018A019D24AD0030
:100E000080302D07CD008A110A12072FCD018A11DB
:100E10000A121D2F5308B4005208B3005108B20043
:100E20005008B10001308A011A21AC01AB008A01DF
:100E30009D24AD0080302D07CD005308B40052082A
:100E4000B3005108B20050088A01ED21AD0032080C
:100E5000AE00AE088A110A12031D382F64302D022D
:100E60008A110A120318382FCE018A110A12482F4C
:100E70005308B4005208B3005108B2005008B10042
:100E800002308A011A21AC01AB008A019D24CE00F8
:100E90000800540855028A110A1203196B2F831691
:100EA0008813831288130830A2002030A90008306C
:100EB000A3004030A4000130AA005408B1008A0108
:100EC000C2205408B1008A01C220831688138312FD
:100ED00088175408D50008008A110A125B1CF42FE9
:100EE0008B135B100610CC01CD01CE01CF0103178F
:100EF0008D01031354088A01AB20831687018312E6
:100F000087018316881183128815831608118312AE
:100F1000081583168810831288148316081083120C
:100F2000081483168701831287010130D408031D3A
:100F30000030003C8A110A12031DAB2FD4038A0132
:100F400049270530DC008A110A16E720D4088A11E7
:100F50000A12031D9E2F0830A2001030A900013094
:100F6000C2008C30C100A601A5012030A100533081
:100F70008A01412069308A01412073308A01412071
:100F800074308A01412065308A0141206D308A0128
:100F9000412020308A0141206B308A01412061309C
:100FA0008A01412070308A01412061308A0141204C
:100FB00074308A01412069308A0141206C308A01F5
:100FC000412064308A01412069308A0141202E305D
:100FD0008A0141200D308A0141200A308A014120D6
:100FE0008B178A150A125D288B133430D400003019
:100FF0008A01A120D6005B140614DB145608D40025
:101000008A01BC253430D4008B17353056028A153E
:101010000A12031812285608D4008A0149278A1593
:101020000A122028D40A8A0149270530DC008A11D7
:101030000A16E720540856028A150A12031D1228C0
:10104000D6010830A2001030A9000130C2008C3057
:10105000C100A601A5012030A10053308A01412022
:1010600069308A01412073308A01412074308A013D
:10107000412065308A0141206D308A0141202030B5
:101080008A01412061308A01412063308A01412078
:1010900069308A0141206C308A01412064308A0124
:1010A000412069308A0141202E308A0141200D30D3
:1010B0008A0141200A308A01412008005B1508306E
:1010C000A2001030A9000130C2008C30C100A6017E
:1010D000A5012030A1004B308A01412075308A01E2
:1010E00041206D308A01412061308A0141206E30FB
:1010F0008A01412064308A01412061308A01412007
:1011000020308A01412074308A01412061308A01F7
:1011100041206E308A01412069308A0141206D30C2
:101120008A01412061308A01412020308A0141201A
:101130006D308A0141206F308A01412064308A017C
:10114000412075308A0141206E308A014120613092
:101150008A01412020308A01412067308A014120E4
:1011600069308A01412072308A01412069308A0148
:1011700041206C308A01412064308A01412069306D
:101180008A0141202E308A0141200D308A01412000
:101190000A308A014120AC010130AB008A019D2454
:1011A000CC00AC011430AB008A019D24CD00CE01EF
:1011B000AC011430AB008A019D24CF008A01FE21CE
:1011C000E6003208E700660A0030031D0130CB005C
:1011D0000301861A01304B048A150A120319DE280E
:1011E0008A150A12861EF7288A110A160828670827
:1011F000E2000830A2001030A9000130C2008C309B
:10120000C100A601A5012030A1004B308A01412078
:1012100075308A0141206D308A01412061308A0198
:1012200041206E308A01412064308A0141206130C2
:101230008A01412020308A01412073308A014120F7
:1012400069308A01412073308A01412074308A015B
:10125000412065308A0141206D308A01412069308A
:101260008A01412020308A0141206F308A014120CB
:101270006B308A01412075308A0141206E308A012D
:10128000412064308A01412075308A0141203A3082
:101290008A01412067088A010F200D308A01412010
:1012A0000A308A014120AC010230AB008A019D2442
:1012B000CC008A01FE21E6003208E700660A003011
:1012C000031D0130CB000301861A01304B048A153F
:1012D0000A12031959298A150A12861E72298A11BF
:1012E0000A1608286608E500620867028A150A12CD
:1012F000031D192A8B130A3003178D000313670887
:101300008A01AB200A308A01E6208B170830A20040
:101310001030A9000130C2008C30C100A601A50127
:101320002030A1004B308A01412075308A014120D4
:101330006D308A01412061308A0141206E308A017E
:10134000412064308A01412061308A0141202030EF
:101350008A01412073308A01412069308A0141208D
:1013600073308A01412074308A01412065308A013E
:1013700041206D308A01412069308A0141202030AE
:101380008A01412064308A0141206F308A01412066
:1013900067308A01412072308A01412075308A010C
:1013A00041206C308A01412061308A0141206E3039
:1013B0008A01412064308A01412069308A0141203C
:1013C00020308A01412076308A01412065308A012F
:1013D000412020308A0141206B308A014120613058
:1013E0008A01412079308A01412064308A014120FC
:1013F00065308A01412064308A01412069308A01C8
:1014000041206C308A01412064308A0141206930DA
:101410008A0141203A308A01412067088A010F2061
:101420000D308A0141200A308A0141208A150A12B2
:10143000C12A0830A2001030A9000130C2008C304F
:10144000C100A601A5012030A1004B308A01412036
:1014500075308A0141206D308A01412061308A0156
:1014600041206E308A01412064308A014120613080
:101470008A01412020308A01412073308A014120B5
:1014800069308A01412073308A01412074308A0119
:10149000412065308A0141206D308A014120693048
:1014A0008A01412020308A01412064308A01412094
:1014B0006F308A01412067308A01412072308A01F1
:1014C000412075308A0141206C308A014120613011
:1014D0008A0141206E308A01412061308A01412019
:1014E0006D308A01412061308A01412064308A01D7
:1014F000412069308A0141202C308A01412020306E
:101500008A01412062308A01412061308A014120F4
:1015100073308A01412074308A01412061308A0190
:1015200041206E308A01412020308A014120623002
:101530008A01412061308A01412073308A014120B3
:101540006C308A01412061308A0141206E308A016D
:10155000412069308A01412079308A0141206F3071
:101560008A01412072308A0141202E308A014120B7
:101570000D308A0141200A308A0141208A150A1261
:101580005E28AC010330AB008A019D24CC008A01A7
:10159000FE21E6003208E700660A0030031D013034
:1015A000CB000301861A01304B048A150A12031975
:1015B000C72A8A150A12861EE02A8A110A160828E6
:1015C000650866028A150A12031D762B8B130530F7
:1015D00003178D00031366088A01AB200A308A01C5
:1015E000E6208B170830A2001030A9000130C2009D
:1015F0008C30C100A601A5012030A10050308A0125
:1016000041206F308A01412077308A0141206530C6
:101610008A01412072308A01412020308A01412014
:1016200074308A01412075308A01412073308A016B
:10163000412075308A01412020308A0141206430E8
:101640008A0141206F308A01412067308A014120A0
:1016500072308A01412075308A0141206C308A0144
:10166000412061308A0141206E308A01412064307E
:101670008A01412069308A01412020308A014120BD
:1016800076308A01412065308A01412020308A016C
:1016900041206B308A01412061308A01412079303C
:1016A0008A01412064308A01412065308A0141204D
:1016B00064308A01412069308A0141206C308A01FE
:1016C000412064308A01412069308A0141203A304A
:1016D0008A01412066088A010F200D308A014120CD
:1016E0000A308A0141208A150A120F2C0830A20004
:1016F0001030A9000130C2008C30C100A601A50144
:101700002030A10050308A0141204F308A01412011
:1017100057308A01412045308A01412052308A01E8
:10172000412020308A01412074308A0141207530E7
:101730008A01412073308A01412075308A0141209D
:1017400020308A01412064308A0141206F308A01B3
:10175000412067308A01412072308A014120753072
:101760008A0141206C308A01412061308A01412088
:101770006E308A01412061308A0141206D308A013A
:10178000412061308A01412064308A014120693062
:101790008A0141202C308A01412020308A014120D9
:1017A00062308A01412061308A01412073308A0110
:1017B000412074308A01412061308A0141206E301D
:1017C0008A01412020308A01412062308A01412073
:1017D00061308A01412073308A0141206C308A01D6
:1017E000412061308A0141206E308A0141206930F8
:1017F0008A01412079308A0141206F308A014120DD
:1018000072308A0141202E308A0141200D308A0138
:1018100041200A308A0141208A150A125E280130CF
:10182000B600F4308A01E720AC010130AB008A0138
:101830009D24CC00AC011530AB008A019D24CD0065
:101840008A01FE21E6003208E700660A0030031D27
:101850000130CB000301861A01304B048A150A12AD
:101860000319202C8A150A12861E392C8A110A1691
:1018700008286608E3000830A2001030A9000130F3
:10188000C2008C30C100A601A5012030A100533058
:101890008A01412065308A01412073308A0141204C
:1018A00020308A0141202B308A01412020308A01DA
:1018B000412062308A01412075308A014120743014
:1018C0008A0141206F308A0141206E308A01412017
:1018D00075308A01412020308A0141206F308A0111
:1018E00041206B308A01412075308A0141206E30E1
:1018F0008A01412064308A01412075308A014120EB
:101900003A308A01412066088A010F200D308A0191
:1019100041200A308A014120AC010230AB008A012B
:101920009D24CC008A01FE21E6003208E700660A09
:101930000030031D0130CB000301861A01304B0437
:101940008A150A120319922C8A150A12861EAB2CCC
:101950008A110A160828630866028A150A12031DEE
:10196000262D8B13063003178D00031366088A019A
:10197000AB200A308A01E6208B170830A200103015
:10198000A9000130C2008C30C100A601A5012030A1
:10199000A10053308A01412065308A014120733013
:1019A0008A01412020308A0141202B308A014120C8
:1019B00020308A01412062308A01412075308A013D
:1019C000412074308A0141206F308A0141206E30FD
:1019D0008A01412075308A01412020308A0141204E
:1019E00076308A01412065308A01412020308A0109
:1019F00041206B308A01412061308A0141207930D9
:101A00008A01412064308A01412065308A014120E9
:101A100064308A01412069308A0141206C308A019A
:101A2000412064308A01412069308A0141203A30E6
:101A30008A01412066088A010F200D308A01412069
:101A40000A308A0141208A150A12C52D0830A200E9
:101A50001030A9000130C2008C30C100A601A501E0
:101A60002030A10053308A01412065308A01412095
:101A700073308A01412020308A0141202B308A01B5
:101A8000412020308A01412062308A014120753096
:101A90008A01412074308A0141206F308A0141203F
:101AA0006E308A01412075308A01412020308A0140
:101AB000412064308A0141206F308A014120673023
:101AC0008A01412072308A01412075308A0141200B
:101AD0006C308A01412061308A0141206E308A01D8
:101AE000412061308A0141206D308A0141206130FE
:101AF0008A01412064308A01412069308A014120F5
:101B00002C308A01412020308A01412062308A0134
:101B1000412061308A01412073308A0141207430B4
:101B20008A01412061308A0141206E308A014120C2
:101B300020308A01412062308A01412061308A01CF
:101B4000412073308A0141206C308A01412061308C
:101B50008A0141206E308A01412069308A0141208A
:101B600079308A0141206F308A01412072308A0128
:101B700041202E308A0141200D308A0141200A3057
:101B80008A0141208A150A125E280130B600F4301D
:101B90008A01E720AC010130AB008A019D24CC0012
:101BA000AC011230AB008A019D24CD008A01FE21D8
:101BB000E6003208E700660A0030031D0130CB0062
:101BC0000301861A01304B048A150A120319D62D17
:101BD0008A150A12861EEF2D8A110A160828660831
:101BE000E4000830A2001030A9000130C2008C309F
:101BF000C100A601A5012030A10053308A01412077
:101C000065308A01412073308A01412020308A01E9
:101C100041202D308A01412020308A01412062304C
:101C20008A01412075308A01412074308A014120A7
:101C30006F308A0141206E308A01412075308A015F
:101C4000412020308A0141206F308A0141206B30D1
:101C50008A01412075308A0141206E308A0141207D
:101C600064308A01412075308A0141203A308A016E
:101C7000412066088A010F200D308A0141200A3078
:101C80008A014120AC010230AB008A019D24CC00C6
:101C90008A01FE21E6003208E700660A0030031DD3
:101CA0000130CB000301861A01304B048A150A1259
:101CB0000319482E8A150A12861E612E8A110A16E9
:101CC0000828640866028A150A12031DDC2E8B138D
:101CD000073003178D00031366088A01AB200A3012
:101CE0008A01E6208B170830A2001030A9000130CD
:101CF000C2008C30C100A601A5012030A1005330E4
:101D00008A01412065308A01412073308A014120D7
:101D100020308A0141202D308A01412020308A0163
:101D2000412062308A01412075308A01412074309F
:101D30008A0141206F308A0141206E308A014120A2
:101D400075308A01412020308A01412076308A0195
:101D5000412065308A01412020308A0141206B30CA
:101D60008A01412061308A01412079308A01412075
:101D700064308A01412065308A01412064308A0143
:101D8000412069308A0141206C308A014120643051
:101D90008A01412069308A0141203A308A0141207C
:101DA00066088A010F200D308A0141200A308A011D
:101DB00041208A150A127B2F0830A2001030A9009A
:101DC0000130C2008C30C100A601A5012030A10065
:101DD00053308A01412065308A01412073308A01E5
:101DE000412020308A0141202D308A0141202030BD
:101DF0008A01412062308A01412075308A014120E8
:101E000074308A0141206F308A0141206E308A018E
:101E1000412075308A01412020308A014120643000
:101E20008A0141206F308A01412067308A014120B8
:101E300072308A01412075308A0141206C308A015C
:101E4000412061308A0141206E308A014120613099
:101E50008A0141206D308A01412061308A01412090
:101E600064308A01412069308A0141202C308A0186
:101E7000412020308A01412062308A0141206130B6
:101E80008A01412073308A01412074308A01412047
:101E900061308A0141206E308A01412020308A0160
:101EA000412062308A01412061308A014120733033
:101EB0008A0141206C308A01412061308A01412031
:101EC0006E308A01412069308A01412079308A01CF
:101ED00041206F308A01412072308A0141202E302A
:101EE0008A0141200D308A0141200A308A014120B7
:101EF0008A150A125E28013003178D000130031382
:101F00008A01AB200830A2001030A9000130C200C5
:101F10008C30C100A601A5012030A10049308A0102
:101F2000412073308A0141206C308A0141206530A4
:101F30008A0141206D308A01412020308A014120F0
:101F400074308A01412061308A0141206D308A015C
:101F5000412061308A0141206D308A0141202C30BE
:101F60008A01412020308A01412062308A014120CB
:101F700069308A0141206C308A01412067308A0132
:101F8000412069308A0141206C308A01412065304E
:101F90008A01412072308A01412020308A0141208B
:101FA0006B308A01412061308A01412079308A01F9
:101FB000412064308A01412065308A01412064302B
:101FC0008A01412069308A0141206C308A01412018
:101FD00064308A01412069308A0141202E308A0113
:101FE00041202E308A0141200D308A0141200A30E3
:101FF0008A0141200B3003178D00013003138A0141
:10200000AB200A308A01E6208A110A160828080047
:102010008B135B100610CC01CD01CE01CF018316CE
:10202000870183128701831688118312881583160E
:1020300008118312081583168810831288148316DA
:102040000810831208148316870183128701203039
:1020500084005C308A01BC20A030840050308A01AA
:10206000BC201030840060308A01BB209030840096
:1020700060308A01BB208A01002863008A110A1699
:102080003D28C3308316810028308B0087018811DA
:102090008312881583160811831208158316881079
:1020A0008312881483160810831208148316881369
:1020B0008312881783160813831208130130D70080
:1020C0008B1706108A110A165B1E72280B30031735
:1020D0008D00003003138A01AB201E308A01E620F8
:1020E0008A016C278A110A16861F81288A110A160E
:1020F000061F81288A110A165B1C81288A150A127C
:102100005E288A110A16DB1D88288A016C27DB11DC
:102110008A110A16DB1EE4288A01FE21E600320835
:10212000E70067085E028A110A16031DE4280A30D8
:10213000DC008A110A16E720660861028A110A1675
:10214000031DB5286430DC008A110A16E7208A01D5
:102150006C278A01BC258A014927FA30DC008A11E4
:102160000A16E7208A110A16E42866085F028A1117
:102170000A16031DCE28540A8A110A160319CB2801
:102180008A110A165B1CCB28D40ADB148A01492762
:102190008A01BC255B178A110A16E42866086002CA
:1021A0008A110A16031DE428D4088A110A16031995
:1021B000E4288A110A165B1CE428D403DB148A0184
:1021C00049278A01BC255B178A110A16722801303B
:1021D0008A01E620DC03DC088A110A16031DE728C1
:0221E0000800F5
:02400E00711E21
:104200005C00000000000000000000000000000052
:084210000000000000000000A6
:00000001FF
